:100000000C9449000C947D000C94BD000C947F016D
:100010000C947F010C947F010C947F010C947F0160
:100020000C947F010C947F010C947F010C947F0150
:100030000C947F010C947F010C947F010C947F0140
:100040000C947F010C947F010C947F010C947F0130
:100050000C947F010C947F010C947F010C947F0120
:100060000C947F010C947F010C947F010C947F0110
:100070000C947F010C947F010C947F010C947F0100
:100080000C947F010C947F010C947F01010001020C
:10009000800011241FBECFEFD0E1DEBFCDBFECE862
:1000A000F0E040E019C0B791A791379127910791EF
:1000B00007FD0EC097918791EF01F92FE82F0BBF35
:1000C00007900D92A217B307D9F7FE011BBE04C01B
:1000D0001D92A217B307E1F7E139F40721F70E9457
:0A00E000FD000C947300F894FFCFAC
:0F00EA003F065B4F666D7D077F6F777C395E79D0
:1000FA001F920F9200905F000F92112400905B00F4
:10010A000F922F933F934F935F936F937F938F93A6
:10011A009F93AF93BF93EF93FF93CF93DF93CDB7A3
:10012A00DEB780910001909101010196909301013F
:10013A008093000180910001909101010E943A018F
:10014A000000DF91CF91FF91EF91BF91AF919F9105
:10015A008F917F916F915F914F913F912F910F9066
:10016A0000925B000F9000925F000F901F9018950D
:10017A001F920F9200905F000F92112400905B0073
:10018A000F922F933F934F935F936F937F938F9326
:10019A009F93AF93BF93EF93FF93CF93DF93CDB723
:1001AA00DEB78091000190910101019790930101BE
:1001BA008093000180910001909101010E943A010F
:1001CA000000DF91CF91FF91EF91BF91AF919F9185
:1001DA008F917F916F915F914F913F912F910F90E6
:1001EA0000925B000F9000925F000F901F9018958D
:1001FA00CF93DF93CDB7DEB70E946B0180E090E02A
:10020A000E943A0181E390E0FC0110828AE690E0C4
:10021A002AE630E0F90120812A60FC01208389E581
:10022A0090E029E530E0F90120812360FC01208378
:10023A0085E390E021E0FC0120837894809100011D
:10024A0090910101892BD1F380E390E0FC01808138
:10025A008330A1F7109201011092000180910001F0
:0A026A00909101010E943A01E9CFD2
:100274000F931F93CF93DF9300D0CDB7DEB79A834C
:10028400898389819A81409724F489819A81992369
:1002940024F48EE090E09A8389830BE310E02AEE45
:1002A40030E040E089819A81092E000CAA0B820F6C
:1002B400931FA41FFC015A2F0E947801862FF80176
:1002C400808300000F900F90DF91CF911F910F91C9
:0202D40008958B
:1002D600CF93DF93CDB7DEB78AE390E02FEFFC0133
:0A02E60020830000DF91CF910895FE
:0E02F00057FD03C05BBF6791089560810895BC
:0402FE000C9400005C
:00000001FF
